:020000040000FA
:1000000001284720831600308500831205158515C9
:1000100011140D089000061B1228111D1228111131
:1000200004309007963093003420930B1428900BE3
:100030000B288316003085008312051185111110DD
:100040008F0B23282D280E08900096309300342023
:10005000930B2728900B2528022883160030850053
:100060008312003085006300920B3B2805141118A1
:10007000851404309200C8308C006430810001087F
:10008000031D3F288C0B3D28051085100034831676
:10009000043081008B13831200308D008E008F009E
:1000A0008C00111004309200831600308500FF3060
:1000B000860083121115061C0230861C0330061DB3
:1000C0000430861D06308D00061E68281830692809
:1000D0000C308E000D088E02861E7628061E7328B0
:1000E00004308F007D2808308F007D28061E7B2875
:1000F00002308F007D2804308F0000349C000511F1
:10010000342034200515342005119C0B812800343F
:00000001FF
